:020000040800F2
:1000000000000220D9040008890A00088B0A0008B1
:100010008D0A00088F0A0008910A000800000000FD
:10002000000000000000000000000000930A00082B
:10003000950A000800000000970A0008990A0008C5
:1000400029050008290500082905000829050008D8
:100050002905000829050008A10A0008290500084B
:1000600029050008AB0A0008290500082905000831
:1000700029050008290500082905000829050008A8
:1000800029050008290500082905000800000000CE
:10009000000000000000000000000000290500082A
:1000A0002905000829050008290500082905000878
:1000B0002905000829050008290500082905000868
:1000C0002905000829050008290500082905000858
:1000D000290500082905000829050008000000007E
:1000E000290500082905000829050008000000006E
:1000F00000000000000000000000000029050008CA
:10010000000000002905000829050008290500084D
:1001100000000000000000000000000000000000DF
:10012000B50A000829050008290500082905000866
:100130002905000800000000000000000000000089
:100140000000000000000000000000002905000879
:1001500029050008290500082905000829050008C7
:100160002905000829050008000000000000000023
:10017000000000000000000000000000000000007F
:100180000000000029050008000000000000000039
:080190002905000829050008FB
:1001980010B5054C237833B9044B13B10448AFF3B9
:1001A80000800123237010BD0C0000200000000017
:1001B800981D000808B5034B1BB103490348AFF36A
:1001C800008008BD0000000010000020981D0008F5
:1001D80053B94AB9002908BF00281CBF4FF0FF31A6
:1001E8004FF0FF3000F072B9ADF1080C6DE904CEA4
:1001F80000F006F8DDF804E0DDE9022304B07047FA
:100208002DE9F047089E04468846002B4BD18A42C8
:10021800154667D9B2FA82F24AB1C2F1200701FA4B
:1002280002F320FA07F7954047EA030894404FEA9B
:10023800154E230CB8FBFEF71FFA85FC0EFB17883A
:1002480043EA084307FB0CF1994209D9EB1807F177
:10025800FF3080F01B81994240F21881023F2B4405
:100268005B1AA4B2B3FBFEF00EFB103344EA03445E
:1002780000FB0CFCA44509D92C1900F1FF3380F0D0
:100288000781A44540F2048102382C4440EA074023
:10029800A4EB0C0400271EB1D4400023C6E9004398
:1002A8003946BDE8F0878B4209D9002E00F0EB8073
:1002B8000027C6E9000138463946BDE8F087B3FA99
:1002C80083F7002F47D18B4202D3824200F2FA8093
:1002D800841A61EB030301209846002EE0D0C6E99A
:1002E8000048DDE702B9FFDEB2FA82F2002A40F0E8
:1002F8008F80491B4FEA154E1FFA85F80127B1FB7D
:10030800FEFC230C0EFB1C1143EA014308FB0CF115
:10031800994207D9EB180CF1FF3002D2994200F24A
:10032800CD808446591AA3B2B1FBFEF00EFB10141F
:1003380043EA044408FB00F8A04507D92C1900F14A
:10034800FF3302D2A04500F2B6801846A4EB080499
:1003580040EA0C409FE7C7F1200CBB4022FA0CFE94
:100368004EEA030E01FA07F420FA0CF521FA0CF311
:100378004FEA1E482543B3FBF8F92C0C08FB193348
:100388001FFA8EFA44EA034309FB0AF49C4202FA74
:1003980007F200FA07F10BD91EEB030309F1FF304E
:1003A80080F087809C4240F28480A9F1020973445E
:1003B8001B1BADB2B3FBF8F008FB103345EA03444E
:1003C80000FB0AFAA24508D91EEB040400F1FF332A
:1003D8006BD2A24569D90238744440EA0940A0FBAF
:1003E8000289A4EB0A044C45C2464B4654D351D06B
:1003F800002E69D0B1EB0A0564EB030404FA0CFC87
:10040800FD40FC404CEA0505C6E90054002747E7D3
:10041800C2F1200320FA03F7954001FA02F021FA0D
:1004280003F34FEA154E3843010CB3FBFEF71FFAEE
:1004380085F80EFB173341EA034107FB08F38B42AB
:1004480004FA02F407D9691807F1FF3C2FD28B424E
:100458002DD9023F2944CB1A81B2B3FBFEF00EFB23
:10046800103341EA034100FB08F38B4207D96918AE
:1004780000F1FF3C17D28B4215D902382944C91A1A
:1004880040EA07473BE73746304609E70746E7E6CD
:100498001846FBE64145ABD2B8EB020A69EB0E02FF
:1004A80001381346A4E76046E9E7184695E767462A
:1004B800D1E781467CE702382C4447E7ACF1020CCF
:1004C8002B442FE7384608E73746E9E6704700BF70
:1004D800DFF834D0002103E00C4B5B584350043163
:1004E8000B480C4B42189A42F6D30B4A02E0002301
:1004F80042F8043B094B9A42F9D300F0DFFA01F0C5
:100508001BFC00F035F9704700000220E01D0008D0
:10051800000000200C0000200C000020EC0000204F
:10052800FEE700002DE9F04188B00024039404940C
:100538000594069407940194264B1A6B42F0010225
:100548001A631A6B02F001020192019A02941A6B63
:1005580042F008021A631B6B03F008030293029B24
:100568001D4E22464FF47041304601F004F9012532
:100578000395DFF86C80CDF810800594174F03A918
:10058800384601F01FF808230393CDF8108005952D
:1005980003A9384601F016F84FF470430393049505
:1005A8000594069403A9304601F00CF8224621462A
:1005B800062000F0A5FD062000F0D6FD22462146C3
:1005C800092000F09DFD092000F0CEFD08B0BDE82F
:1005D800F08100BF00380240000C024000000240D9
:1005E8000000111000B583B000210191094B1A6B6E
:1005F80042F480021A631B6B03F480030193019B8E
:100608000A46382000F07CFD382000F0ADFD03B02C
:100618005DF804FB0038024070B584B000230093F5
:10062800019302930393184C184A22604FF4403206
:100638006260A36001252561257684F82030E36295
:10064800134AA262E3600326E66184F830506561CC
:10065800204600F057FB0095019507230293694651
:10066800204600F069FC0223009301936946204666
:1006780000F062FC074B009301966946204600F0A3
:100688005BFC04B070BD00BF3800002000200140B2
:100698000100000F1200001010B50446082802D00F
:1006A800012C11D010BD0821104801F05DF8002878
:1006B800F6D10F4B1B781BB90D4B01221A70EFE7CF
:1006C8000B4B00221A70EBE70121084801F04CF8A7
:1006D8000128E7D1064B5B78DBB2012BE2D1044B52
:1006E80000225A7001229A70DCE700BF0000024025
:1006F8002800002010B594B03022002108A801F08D
:100708003FFB0024039404940594069407940194F1
:10071800154B1A6C42F080521A641B6C03F080531C
:100728000193019B0294114B1A6842F440421A60EB
:100738001B6803F440430293029B0223089301239E
:100748000B9310230C930E9408A801F029F80F239B
:1007580003930494059406940794214603A801F092
:100768003FFA14B010BD00BF0038024000700040CE
:1007780008B500F0EDF9FFF7BDFFFFF7D3FEFFF76F
:1007880031FFFFF749FF032279497A4800F0E6FA7A
:1007980075E0794C01224FF40041204600F0EBFF50
:1007A80001224FF48051204600F0E5FF01224FF46A
:1007B8000051204600F0DFFF01224FF4804120461F
:1007C80000F0D9FFA62000F0EFF900224FF4004115
:1007D800204600F0D0FF00224FF48051204600F060
:1007E800CAFF00224FF40051204600F0C4FF002247
:1007F8004FF48041204600F0BEFFA62000F0D4F957
:100808005B4B9A885D4B1A801B889BB207EE903A27
:10081800F8EEE77ADFED5A6A87EEA67AF0EE087A04
:1008280067EE277A574BC3ED007A93ED007ADFED38
:10083800567A37EE677ADFED556AC7EE267AB3EE59
:10084800097A77EE877A524BC3ED007A93ED007AF6
:10085800F3EE0E7AB4EEE77AF1EE10FA05DD4D4BC1
:100868009B7813B94B4B01225A70494B93ED007A90
:10087800F3EE0E7AB4EEE77AF1EE10FA73D9454B3F
:100888005B78002B85D13A4B1B88B3F5806F02D279
:10089800404A127812B3B3F5406F03D33D4A127839
:1008A800012A1BD0B3F5406F03D33A4A1278002AC5
:1008B80044D0B3F5806F03D2364B1B78012B3DD063
:1008C8002D4C00224FF40041204600F054FF002236
:1008D8004FF40051204600F04EFF05E001224FF48E
:1008E8000041254800F047FF214B5B88B3F5806F36
:1008F80002D2284A127842B3B3F5406F03D3254A8F
:100908001278012A21D0B3F5406F02D3214A127818
:1009180012B3B3F5806F03D21E4B1B78012B1BD08B
:10092800154C00224FF48051204600F024FF00228D
:100938004FF48041204600F01EFF61E701224FF48A
:1009480000510D4800F017FFCEE701224FF4805107
:10095800094800F010FF53E701224FF48041064890
:1009680000F009FF4CE70B4B00229A7087E700BFA5
:10097800E000002038000020000C02402C0000207D
:1009880000F07F45300000205C8F423F0AD7233BB0
:1009980034000020280000207047000082B00021A9
:1009A80000910B4B5A6C42F480425A645A6C02F420
:1009B80080420092009A01911A6C42F080521A64A7
:1009C8001B6C03F080530193019B02B0704700BF7A
:1009D8000038024030B589B000230393049305938F
:1009E80006930793026803F1804303F590339A4214
:1009F80001D009B030BD04460025019503F58C33BC
:100A08005A6C42F480725A645A6C02F480720192F1
:100A1800019A02951A6B42F001021A631B6B03F0EC
:100A280001030293029B062303930323049303A960
:100A3800104800F0C7FD1048104B03604560856002
:100A4800C5604FF4806303614FF4006343614FF462
:100A5800005383614FF48073C3610562456200F0FF
:100A680023FC18B9044BA3639C63C2E7FFF794FF08
:100A7800F8E700BF00000240800000201064024038
:100A88007047FEE7FEE7FEE7FEE7704770477047EE
:100A980008B500F077F808BD08B5012000F072FE2F
:100AA80008BD08B5082000F06DFE08BD08B502486D
:100AB80000F09AFC08BD00BF800000200F49D1F863
:100AC800883043F47003C1F888300D4B1A6842F03F
:100AD80001021A60002098601A6822F0847222F4D9
:100AE80080321A60074A5A601A6822F480221A6013
:100AF800D8604FF000638B60704700BF00ED00E0E6
:100B0800003802401030002410B504460E4B187807
:100B18004FF47A73B3FBF0F30C4A1068B0FBF3F0B0
:100B280000F030FB68B90F2C01D901200AE000223F
:100B380021464FF0FF3000F0E3FA034B5C600020E1
:100B480000E0012010BD00BF0400002000000020CC
:100B580008B50B4B1A6842F400721A601A6842F41E
:100B680080621A601A6842F480721A60032000F0EA
:100B7800B5FA0020FFF7C8FFFFF710FF002008BDF7
:100B8800003C0240034A1168034B1B780B44136076
:100B9800704700BFE800002004000020014B1868DF
:100BA800704700BFE800002038B50446FFF7F6FF9D
:100BB8000546B4F1FF3F02D0044B1B781C44FFF7F5
:100BC800EDFF401BA042FAD338BD00BF040000204F
:100BD8004A4B5A6822F440325A605A6841680A43BC
:100BE8005A600268536823F480735360026853683C
:100BF800016943EA012353600268536823F0407394
:100C080053600268536881680B43536002689368B5
:100C180023F40063936002689368C1680B43936090
:100C2800826A374B9A424BD00268936823F070630C
:100C3800936002689368816A0B43936002689368C3
:100C480023F04053936002689368C16A0B43936032
:100C58000268936823F00203936002689368017E38
:100C680043EA4103936090F82030002B33D10268A7
:100C7800536823F4006353600268D36A23F4700353
:100C8800D3620168CB6AC269013A43EA0253CB6274
:100C98000268936823F4007393600268936890F87D
:100CA800301043EA412393600268936823F4806319
:100CB800936002689368416943EA812393607047AF
:100CC8000268936823F0706393600268936823F066
:100CD80040539360BCE70268536843F40063536071
:100CE8000268536823F46043536001684B68426AA2
:100CF800013A43EA42334B60BEE700BF002301409C
:100D08000100000F38B310B50446036C43B1236CDF
:100D180013F0100F0BD00120002384F83C3010BDD5
:100D2800FFF758FE0023636484F83C30EFE7236C38
:100D380023F4885323F0020343F00203236420467C
:100D4800FFF746FF00206064236C23F0030343F0A1
:100D580001032364E0E701207047000030B583B049
:100D68000023019390F83C30012B00F0818001238F
:100D780080F83C300468A36813F0010F13D1A3680E
:100D880043F00103A3603F4B1C683F4BA3FB0434B3
:100D9800A40C04EB4404019402E0019C013C01947E
:100DA800019C002CF9D103689C6814F0010F61D0F4
:100DB800046C24F4E06424F0010444F480740464B2
:100DC8005B6813F4806F05D0036C23F4405343F43D
:100DD80080530364036C13F4805F36D0436C23F0B4
:100DE8000603436413460446002280F83C20826BC5
:100DF8002648D063A26B26481064A26B2548D064AD
:100E080022686FF0220010602568686840F08060F2
:100E180068602568A86840F48070A86020680A4661
:100E280000F14C01A06B00F0A5FA1B4B5B6813F0B6
:100E38001F0F0DD123689A6812F0405F1DD19A6880
:100E480042F080429A60002015E000234364C9E71D
:100E58002368124A934201D000200CE09A6812F0ED
:100E6800405F0CD19A6842F080429A60002002E00C
:100E7800022000E0002003B030BD0020FBE7002086
:100E8800F9E700BF0000002083DE1B43CF0E0008F7
:100E9800AD0E0008B90E00080023014000200140F3
:100EA8007047704708B5806BFFF7FBFF08BD7047B8
:100EB80008B5806B40230364436C43F00403436428
:100EC800FFF7F5FF08BD08B5836B1A6C12F0500FD9
:100ED80026D11A6C42F400721A641A68916811F0EB
:100EE800405F19D1197EB9B9D16A11F4700F03D0D6
:100EF800916811F4806F0FD1516821F02001516081
:100F08001A6C22F480721A641A6C12F4805F03D18E
:100F18001A6C42F001021A641846FFF7C1FF08BDB7
:100F28001A6C12F0100F03D19B6BDB6C9847F6E735
:100F38001846FFF7BCFFF2E730B482B000230193F4
:100F480090F83C30012B00F0BD80012380F83C3044
:100F58000B68092B3ED90568EA689BB203EB43038B
:100F68001E3B072404FA03F322EA0303EB60056837
:100F7800EA688C680B8803EB43031E3B04FA03F30F
:100F88001343EB604B68062B3AD805686A6B03EB92
:100F98008303053B1F2404FA03F322EA03036B636C
:100FA80005686A6B4B6803EB8303053B0C8804FAFE
:100FB80003F313436B630268434B9A4250D00268B1
:100FC800414B9A4259D0002380F83C30184602B071
:100FD80030BC704705682A699BB203EB43030724BA
:100FE80004FA03F322EA03032B6105682A698C6873
:100FF8000B8803EB430304FA03F313432B61C1E7A4
:101008000C2B16D805682A6B03EB8303233B1F249C
:1010180004FA03F322EA03032B6305682A6B4B687F
:1010280003EB8303233B0C8804FA03F313432B637A
:10103800C1E70568EA6A03EB8303413B1F2404FA0E
:1010480003F322EA0303EB620568EA6A4B6803EBE1
:101058008303413B0C8804FA03F31343EB62AAE7CA
:101068000B68122BABD1194B5A6822F400025A6054
:101078005A6842F480025A60A1E70B68144A934206
:1010880001D0112B9FD1114B5A6822F480025A606B
:101098005A6842F400025A600A680D4B9A4292D18B
:1010A8000C4B1B680C4AA2FB03239B0C03EB83032A
:1010B8005A00019202E0019B013B0193019B002B26
:1010C800F9D180E7022082E7002001400023014097
:1010D800120000100000002083DE1B43074AD3687B
:1010E80023F4E0631B041B0C000200F4E0601843C7
:1010F80040F0BF6040F40030D060704700ED00E081
:1011080030B4174BDB68C3F30223C3F10704042C84
:1011180028BF04241D1D062D18D9033B4FF0FF35A9
:1011280005FA04F421EA0401994005FA03F322EAD6
:101138000303194300280BDB0901C9B200F1604021
:1011480000F5614080F8001330BC70470023E5E7E4
:1011580000F00F000901C9B2024B1954F4E700BFAF
:1011680000ED00E014ED00E0002807DB00F01F02AE
:10117800400901239340024A42F82030704700BFDB
:1011880000E100E00138B0F1807F0AD2064B5860D8
:10119800064AF02182F823100020986007221A607E
:1011A80070470120704700BF10E000E000ED00E04C
:1011B80030B405682C6824F480242C6004686360CB
:1011C8008368402B05D0036899600368DA6030BCF7
:1011D800704703689A600368D960F8E70268D3B279
:1011E800103B0B49A1FB03131B090A49C95CC165E4
:1011F800032B06D822F47F7222F003028265806DE9
:10120800704722F47F7222F0030204328265F6E707
:10121800ABAAAAAAC81D0008836A826992B9012BE1
:101228000AD01BB1022B01D000207047C36A13F00B
:10123800807F2CD100207047C36AB3F1C07F28D0CB
:1012480000207047B2F5005F05D0022B29D9032B87
:1012580015D000207047032B03D8DFE803F01C04E7
:101268001C0A00207047C36A13F0807F15D1002044
:101278007047C36AB3F1C07F11D000207047C36ABA
:1012880013F0807F01D001207047002070470120B3
:1012980070470120704701207047012070470120E6
:1012A800704701207047000070B50446FFF776FCD0
:1012B800002C5BD00546002384F83430022384F8E0
:1012C80035302268136823F00103136023681A6815
:1012D80012F0010F0AD0FFF761FC401B0528F5D971
:1012E80020236365032084F8350070BD1A68204800
:1012F80010406168A2680A43E1680A4321690A4309
:1013080061690A43A1690A43E1690A43216A0A43F8
:101318000243616A04291ED01A602668756925F09F
:101328000705636A1D43042B07D1A36A1D43E36ABB
:101338001BB12046FFF770FF90B975612046FFF793
:101348004DFFE26D3F2393408360002060650123D9
:1013580084F83530C9E7E16A206B01430A43DBE7CB
:1013680040236365012084F83500BEE70120BCE70F
:101378003F8010F038B5856D90F83440012C31D09D
:10138800012480F8344090F83540E4B2012C04D0B0
:10139800002380F83430022038BD0446022084F847
:1013A8003500002060652046FFF702FFE26D3F230D
:1013B8009340AB602268136843F0160313602268F9
:1013C800536943F080035361236C23B12268136887
:1013D80043F0080313602268136843F001031360A5
:1013E8000020D9E70220D7E7F0B583B004460023F0
:1013F8000193724B1D68724BA3FB0535AD0A876DCF
:101408003E68C26D08239340334210D003681A68BF
:1014180012F0040F0BD01A6822F004021A60C26D91
:1014280008239340BB60436D43F001034365E26DBD
:1014380001239340334209D02268526912F0800F89
:1014480004D0BB60636D43F002036365E26D04235F
:101458009340334209D02268126812F0020F04D078
:10146800BB60636D43F004036365E26D1023934032
:10147800334224D02268126812F0080F1FD0BB60D4
:1014880023681A6812F4802F0DD01B6813F4002FFC
:1014980004D1236C9BB12046984710E0A36C73B12C
:1014A800204698470BE01A6812F4807F03D11A6827
:1014B80022F008021A60236C0BB120469847E26DAF
:1014C80020239340334255D02268126812F0100F3F
:1014D80050D0BB6094F83530DBB2052B0ED02368B2
:1014E8001A6812F4802F33D01B6813F4002F2AD106
:1014F800636C002B3ED0204698473BE02268136877
:1015080023F0160313602268536923F080035361A4
:10151800236CA3B12268136823F008031360E26DFB
:101528003F239340BB60002384F83430012384F8C0
:101538003530236D002B3FD0204698473CE0A36C04
:10154800002BE7D1EBE7E36BA3B12046984711E006
:101558001A6812F4807F09D11A6822F010021A6002
:10156800002384F83430012384F83530E36B0BB161
:1015780020469847636DFBB1636D13F0010F17D0D8
:10158800052384F835302268136823F001031360BB
:10159800019B01330193AB4204D823681B6813F005
:1015A800010FF5D1002384F83430012384F8353055
:1015B800E36C0BB12046984703B0F0BD0000002053
:1015C800B5814E1B00230F2B00F2C580F0B482B00A
:1015D80039E0042200E00022B2403A4302345E4E71
:1015E80046F824205D4A1468EA4302EA04064F6874
:1015F80017F4803F01D045EA0406584C2660646819
:1016080002EA04064F6817F4003F01D045EA0406D1
:10161800524C6660A46802EA04064F6817F4801FFB
:1016280001D045EA04064D4CA660E46822404E68A5
:1016380016F4001F01D045EA0402484CE260013369
:101648000F2B00F2858001229A400C6804EA0205FB
:10165800AA42F4D14C68022C01D0122C10D1DE0819
:10166800083650F826C003F00704A7000F24BC4032
:101678002CEA040C0C69BC4044EA0C0440F82640EF
:1016880004685F000326BE40F64306EA040C4C6873
:1016980004F00304BC4044EA0C0404604C6804F100
:1016A800FF3CBCF1010F03D9112C01D0122C10D131
:1016B800846806EA040CCC68BC4044EA0C048460E4
:1016C800446824EA02024C68C4F300149C401443A2
:1016D8004460C26816408A68BA403243C2604A68A9
:1016E80012F0805FABD0002201921D4A546C44F482
:1016F80080445464526C02F480420192019A9C081E
:10170800A61C154A52F8267003F0030296000F2211
:10171800B24027EA0207134A90423FF45CAF02F551
:10172800806290420ED002F5806290420CD002F5A1
:10173800806290420AD002F5806290423FF449AF3D
:10174800072249E7012247E7022245E7032243E748
:1017580002B0F0BC7047704700380140003C0140BF
:1017680000380240000002400369194201D10020FC
:1017780070470120704712B909048161704781617F
:101788007047000008B5054B5B69034200D108BDEE
:10179800024B5861FEF780FFF9E700BF003C0140AB
:1017A800002800F0BB8170B582B00446036813F0CE
:1017B800010F3BD0A74B9B6803F00C03042B2CD0E4
:1017C800A44B9B6803F00C03082B21D06368B3F586
:1017D800803F4FD0B3F5A02F52D09E4B1A6822F409
:1017E80080321A601A6822F480221A606368002B1B
:1017F80050D0FFF7D3F90546964B1B6813F4003F0A
:1018080014D1FFF7CBF9401B6428F5D903208AE1EE
:10181800904B5B6813F4800FD8D08E4B1B6813F481
:10182800003F03D06368002B00F07A81236813F02F
:10183800020F55D0874B9B6813F00C0F3ED0854B99
:101848009B6803F00C03082B33D0E368002B68D0A7
:10185800814B01221A60FFF7A1F905467D4B1B68F1
:1018680013F0020F54D1FFF799F9401B0228F5D95C
:10187800032058E1774A136843F480331360B5E7CF
:10188800744B1A6842F480221A601A6842F4803253
:101898001A60ABE7FFF782F905466E4B1B6813F435
:1018A800003FC3D0FFF77AF9401B6428F5D903201D
:1018B80039E1684B5B6813F4800FC6D1654B1B6830
:1018C80013F0020F04D0E368012B01D001202AE1B4
:1018D800604A136823F0F803216943EAC1031360DF
:1018E800236813F0080F40D0636963B35B4B012290
:1018F8001A60FFF753F90546564B5B6F13F0020F5A
:1019080033D1FFF74BF9401B0228F5D903200AE130
:10191800504A136823F0F803216943EAC1031360AE
:10192800DEE74D4B00221A60FFF738F90546494BB0
:101938001B6813F0020FD3D0FFF730F9401B0228C1
:10194800F5D90320EFE0454B00221A60FFF726F98E
:101958000546404B5B6F13F0020F06D0FFF71EF9E8
:10196800401B0228F5D90320DDE0236813F0040F9B
:1019780079D0384B1B6C13F0805F33D1002301936F
:10198800344B1A6C42F080521A641B6C03F080537B
:101998000193019B0125324B1B6813F4807F23D0F0
:1019A800A368012B34D0052B38D02A4B1A6F22F0AC
:1019B80001021A671A6F22F004021A67A368002B43
:1019C80036D0FFF7EBF80646224B1B6F13F0020FD9
:1019D80048D1FFF7E3F8801B41F288339842F3D9E6
:1019E8000320A0E00025D6E71D4A136843F480735E
:1019F8001360FFF7D3F80646194B1B6813F4807F72
:101A0800CED1FFF7CBF8801B0228F5D903208AE056
:101A1800104A136F43F001031367CFE70D4B1A6F9A
:101A280042F004021A671A6F42F001021A67C5E70A
:101A3800FFF7B4F80646074B1B6F13F0020F11D0DF
:101A4800FFF7ACF8801B41F288339842F3D90320A2
:101A580069E000BF0038024000004742800E47425C
:101A680000700040E5B9A369002B5BD0304A92684A
:101A780002F00C02082A58D0022B17D02D4B002256
:101A88001A60FFF78BF80446294B1B6813F0007F98
:101A980042D0FFF783F8001B0228F5D9032042E063
:101AA800234A136C23F080531364DCE7214B002294
:101AB8001A60FFF773F805461D4B1B6813F0007F8B
:101AC80006D0FFF76BF8401B0228F5D903202AE05F
:101AD800E369226A1343626A43EA8213A26A5208DC
:101AE800013A43EA0243E26A43EA0263104A536056
:101AF800104B01221A60FFF751F804460C4B1B6883
:101B080013F0007F06D1FFF749F8001B0228F5D92A
:101B1800032008E0002006E0002004E001207047D0
:101B2800012000E0002002B070BD0120FBE700BFEB
:101B38000038024060004742264B9B6803F00C03C4
:101B4800042B44D0082B01D0234870472DE9F04BD3
:101B5800204B5A6802F03F025B6813F4800F13D0E1
:101B68001C4B5968C1F3881100231C48A1FB0001D4
:101B7800FEF72EFB174B5B68C3F3014301335B0091
:101B8800B0FBF3F0BDE8F08B124B5B68C3F388132E
:101B98001E4600275C010025E41A65EB0705A9012C
:101BA80041EA9461A001001B61EB0501CB0043EA07
:101BB8005073C400A01943EB07018B0243EA90530A
:101BC8008402204619460023FEF702FBD2E70348A9
:101BD800704700BF003802400024F40040787D01BF
:101BE800002800F09D8070B504464F4B1B6803F039
:101BF8000F038B4209D2CBB24B4A1370136803F020
:101C08000F038B4201D0012070BD236813F0020F2F
:101C180017D013F0040F04D0444A936843F4E053F8
:101C28009360236813F0080F04D0404A936843F484
:101C3800604393603D4A936823F0F003A068034330
:101C480093600D46236813F0010F32D06368012BAF
:101C580021D09A1E012A25D9344A126812F0020F9F
:101C680060D032498A6822F0030213438B60FEF782
:101C780095FF06462D4B9B6803F00C036268B3EB97
:101C8800820F16D0FEF78AFF801B41F288339842F4
:101C9800F0D90320B8E7254A126812F4003FE0D1D2
:101CA8000120B1E7214A126812F0007FD9D1012042
:101CB800AAE71D4B1B6803F00F03AB4209D9EAB230
:101CC800194B1A701B6803F00F03AB4201D00120B7
:101CD8009AE7236813F0040F06D0144A936823F494
:101CE800E053E1680B439360236813F0080F07D0B3
:101CF8000E4A936823F46043216943EAC103936061
:101D0800FFF71AFF094B9B68C3F30313084AD35C18
:101D1800D840084B18600020FEF7F6FE002073E755
:101D28000120704701206FE7003C02400038024064
:101D3800B01D00080000002070B50D4E0D4CA41B0E
:101D4800A4100025A54209D10B4E0C4C00F020F838
:101D5800A41BA4100025A54205D170BD56F8253056
:101D680098470135EEE756F8253098470135F2E7F0
:101D7800D81D0008D81D0008D81D0008DC1D000863
:101D880002440346934200D1704703F8011BF9E768
:101D9800F8B500BFF8BC08BC9E467047F8B500BF50
:081DA800F8BC08BC9E46704720
:101DB00000000000000000000102030406070809FB
:101DC00000000000010203040006101600061016B1
:081DD00038E4FF7F0100000070
:041DD800BD01000841
:041DDC009901000861
:0C1DE0000024F4000100000010000000CE
:04000005080004D912
:00000001FF
